:10019B003F065B4F666D7D077F6F777C395E7971AC
:0701BB00AE071FEE70FA22EF
:03002B00020003CD
:10000300C0E0C0D0C2CFE509C39508400AE5099412
:100013000A5004D2B68002C2B60509E509B40A0340
:08002300750900D0D0D0E032D5
:10015700EF24FE600B14600C2402700AD2028006A2
:10016700D2008002B20130021130010E0508C2022E
:10017700E508C3940A4003E4F50830000F30010C8A
:100187001508C200E508B4FF03750809200104C279
:0401970002C200227E
:10010F0075CDB175CCE075CBB175CAE0D2AFD2ADBC
:10011F00D2CA1201AB30031D1200BA8F0AEF900141
:10012F009B93F4F58075A0FE7FC81201BBAF0A1236
:10013F000157E4F50AE50890019B93F4F58075A04B
:08014F00FD7FC81201BB80CA4C
:0201CF00C1036A
:0701C200AE071FEE70FA22E8
:0601C900EF25E0FF0F220C
:0F01AB007590F0AF90EF64F06003D20322C203AF
:0101BA002222
:1000BA0079017CFE7BEF1201AB300346C2037FC895
:1000CA001201C21201AB300339E4FE8C90E4FAAF9C
:1000DA00905307F0EB54F0F50BB5070D30030512FA
:1000EA0001AB80F8AD01AF052209AF031201C9AB1C
:1000FA00070ABA04DA7BEFAF041201C9AC070EBED5
:04010A0004C9AF0570
:01010E0022CE
:0300000002002ECD
:0C002E00787FE4F6D8FD75812002007593
:10003A0002010FE493A3F8E493A34003F68001F2CC
:10004A0008DFF48029E493A3F85407240CC8C333C7
:10005A00C4540F4420C8834004F456800146F6DF96
:10006A00E4800B01020408102040809001CFE47E56
:10007A00019360BCA3FF543F30E509541FFEE4938B
:10008A00A360010ECF54C025E060A840B8E493A352
:10009A00FAE493A3F8E493A3C8C582C8CAC583CA7D
:1000AA00F0A3C8C582C8CAC583CADFE9DEE780BE35
:0101D100002D
:00000001FF
